:100000000C94230C0C944B0C0C944B0C0C944B0C3C
:100010000C944B0C0C944B0C0C944B0C0C942A3100
:100020000C944B0C0C944B0C0C944B0C0C944B0CF4
:100030000C944B0C0C944B0C0C9417350C944B0CEF
:100040000C944D350C944B0C0C9410370C94623777
:100050000C944B0C0C9465300C944B0C0C944B0C86
:100060000C9434330C944B0CB4000000FF000000DF
:100070000000C800FF03FF00FF000700FF00FF00B3
:10008000000608100A07FFFFFDF7EDF304FA0EDA89
:10009000B1A99FA5A29EA4AAA2A6978BA4C6D8E5A3
:1000A000E8F700000C151C202A333E48463A2A1F68
:1000B0001205FDF8F2EBE6DED8D0CDC2BCC9D7E41C
:1000C000EEF7010B0F141B222931393E484E4F49E0
:1000D0003D2E1F0F03F8F1ECE4DCD4CFC9C4BFBD43
:1000E000B4B0BED0E0EDF6010B111821292F363B3C
:1000F00040454B5358574F4132221305F9EEE5DF87
:10010000D8D1CBC6C1BDB9B6B3B2ADAFC0D3E3F0A1
:10011000FA0610171F272E343B4144484D51545ABC
:100120005D5A53473A2A1B0BFDF1E7DED8D1CBC409
:10013000BFBBB8B5B2AFADACACADACB4C7DAEAF7E3
:10014000020E171E262E353B42474A4E5155585B2C
:100150005C5D5F5F5A51453829190AFDF2E7DDD42D
:10016000CDC7C1BDB8B3AEABA9A8A7A6A5A5A5A785
:10017000ABACB5C8DBEBF7020D161D252C343B42AA
:10018000464A4E5256595C5D5D5D5E5E605F5A51F7
:10019000463A2E211305F7EBE0D7CEC5BEB8B2AE76
:1001A000A9A6A29F9C9B9B9B9C9D9FA1A3A6AAAE38
:1001B000B2B6C1D5E7F6020B151C232A31383F45EC
:1001C0004A4F53575B5F6264656566666666656342
:1001D00062605A52493D32261A0E02F6EADFD4CA4C
:1001E000C2B9B2ABA5A09B989592908E8D8D8F9041
:1001F0009396999CA0A4A8ACB0B5BABFC5D4E6F7B5
:10020000040E1720272D343A41494F55595E626636
:10021000696C6D6E6F6F6F6E6D6B69676563626041
:100220005C5750483F362B21170D03F8EDE2D7CD30
:10023000C4BBB3ABA39D97928F8C89878685858538
:100240008586888A8C8F9296999C9FA2A5A8ACB02F
:10025000B4B8BDC2CDDFF0FF0B151F282F363E45C9
:100260004D545B61676C7175797B7C7D7D7D7D7D97
:100270007B79777472706D6B686663615E59534CFD
:10028000443B32291F150C02F8EEE4DACFC5BCB3AB
:10029000AAA39B958F8B87848281808080828385AF
:1002A000878A8C8E9194979A9DA1A4A7ABAEB1B486
:1002B000B7BABDC0C4C7CCD1D6DFECFA08131D2530
:1002C0002C33383E444A50565A5F63686C6F7273E1
:1002D00074757575757473727170706F6E6C6B690F
:1002E000676664625F5C5956524D47403830292139
:1002F00019100800F8F0E8E0D8D0C8C0B9B2ABA433
:100300009F9994908D8A888785858585858687883D
:10031000898B8C8F90929395989A9D9FA2A5A7AA5E
:10032000ACAFB1B4B6B8BBBDC0C4C9CED6E0EDFA6F
:1003300006111A232A31373E454B51575C61666BD3
:100340006F7376787A7C7D7E7E7E7D7C7C7B7A790D
:10035000777675747371706E6C6A6765625F5B57F0
:10036000534F4A453F39322B241D150E06FFF8F036
:10037000E9E2DBD3CCC5BEB8B1ABA59F9994908C14
:100380008885838280808080808182848587898B34
:100390008D8F91939596999B9EA0A3A6A9ACAFB281
:1003A000B5B7BBBEC1C4C7CBCED3D8DEE5EEF8032C
:1003B0000E171F272E343A3F454A5054595D616548
:1003C000686B6E70727475767777777676757574FC
:1003D0007372716F6E6D6C6A696664615E5B5753B0
:1003E000504C47433F3B36312C27221C17110B053D
:1003F00000FAF5EFEAE4DFDAD5D0CBC6C1BCB8B37A
:10040000AFAAA6A29E9B9896949291908F8F8F8F61
:1004100090909193949597999B9D9FA1A4A6A7A92D
:10042000ACAEB1B3B6B9BCBFC1C4C7C9CCCFD2D5CD
:10043000D8DBDFE3E8EDF4FB040E171F272E343979
:100440003F44494D5156595D606366696B6C6E6FF0
:1004500070717171717170706F6E6D6C6B6A6867BD
:10046000656462605E5C5A5753504C4844403C3867
:1004700034302C28241F1B17120D0904FFFAF5F045
:10048000ECE7E2DEDAD5D1CDC9C5C1BEBAB6B3AFAD
:10049000ACA8A6A3A09E9C9A999796969595969699
:1004A0009798999A9C9E9FA1A3A5A7AAACAEB0B21B
:1004B000B4B6B9BCBFC1C4C7CACDCFD2D5D8DBDDB5
:1004C000E0E4E7EAEEF2F7FD040B131B232A3137D1
:1004D0003C41464A4E5255595C5F61646667696AA1
:1004E0006A6B6B6B6B6B6B6A6A6968676564636187
:1004F0005F5E5C5A575553504E4B4744403C38342E
:10050000302C2824201C1814110D090501FDF9F5C3
:10051000F1EDE9E6E2DEDBD7D4D1CECAC7C4C1BE75
:10052000BCB9B6B3B1AEACAAA8A6A5A3A2A1A09F20
:100530009F9F9FA0A0A1A2A4A5A7A9AAACAEB1B35A
:10054000B5B7B9BCBEBFC2C4C7CACCCFD2D5D7DA43
:10055000DDDFE2E5E8EAEDF0F3F7FAFE03090F1656
:100560001C232A30353B4044484C505356595B5E5F
:10057000606163646565666666656564646362613F
:100580005F5E5C5A585654524F4D4A4744423F3C76
:100590003835312D2925211D1A16130F0C09060394
:1005A00000FDFAF7F4F0EDEAE7E4E1DEDBD9D6D3BB
:1005B000D1CECCC9C7C5C2C0BEBBB9B7B5B4B2B144
:1005C000B0AEADACABABAAAAAAAAABACADAEAFB164
:1005D000B2B4B5B7B9BBBDBFC1C3C6C8C9CBCDCF17
:1005E000D2D4D7DADCDFE1E4E6E9EBEEF0F3F5F8BC
:1005F000FBFE02060A0F141A20252B30353A3E4224
:1006000046494D50525557595B5C5D5E5F5F5F5F79
:100610005F5E5E5D5C5B5A58565553504E4C494682
:1006200043413E3B3835322F2C2825211D1A171304
:10063000100D0A070402FFFDFBF8F6F3F1EEECE9FA
:10064000E7E4E2E0DDDBD9D7D4D2D0CECCCAC8C74C
:10065000C5C3C1BFBEBCBBBAB9B8B7B6B6B5B5B4F1
:10066000B4B5B5B6B7B7B9BABBBDBEC0C2C4C5C7CD
:10067000C9CBCDCFD1D2D4D6D8DADDDFE2E4E6E9FA
:10068000EBEDEFF2F4F6F8FBFD0003060A0E12178D
:100690001B20252A2E32363A3E4144474A4C4E50C2
:1006A00052545556565757575757565555545251F9
:1006B0004F4D4B494644413E3B393633302D2A2875
:1006C00025221E1B1815120F0C0A07050200FEFC3E
:1006D000FAF8F6F4F2F0EEECEAE8E6E4E1E0DEDC6B
:1006E000DAD8D6D4D3D1CFCECCCAC9C7C6C5C4C236
:1006F000C2C1C0BFBFBEBEBDBDBDBEBEBFC0C1C208
:10070000C3C4C6C7C9CACCCDCFD1D3D4D6D7D9DA02
:10071000DCDFE1E3E5E7E9EBEEEFF1F4F5F8FAFC15
:10072000FE000205080B0E12161A1E2226292D3075
:1007300034373A3D3F42444648494A4B4C4D4D4E72
:100740004E4E4D4D4C4B4A4947464442403D3B3846
:100750003633302E2B282624211F1C191614110E77
:100760000C0A07050301FFFEFCFAF9F7F5F4F2F0B5
:10077000EEECEAE9E7E5E3E1E0DEDDDBD9D8D6D56A
:10078000D3D2D1CFCECDCCCBCAC9C8C8C7C6C6C6B6
:10079000C5C5C5C6C6C7C8C8C9CBCCCDCED0D1D3B8
:1007A000D4D6D8D9DBDDDEDFE1E3E5E7E9EBEDEF39
:1007B000F0F2F4F6F7F9FBFCFEFF01030507090B65
:1007C0000E111316181B1D1F2123252728292B2C3A
:1007D0002D2D2E2F2F2F2F2F2F2E2E2D2D2C2B2A40
:1007E000292827252422201F1D1C1A18171514122A
:1007F00011100E0D0B0A0907060504030201000083
:10080000FFFEFEFDFCFCFBFBFAF9F9F8F7F7F6F644
:10081000F6F5F5F4F4F4F3F3F3F3F3F2F2F2F2F2A3
:10082000F2F2F2F2F2F2F3F3F3F3F4F4F4F5F5F595
:10083000F6F6F7F7F8F8F9F9F9FAFAFBFBFBFCFC26
:10084000FCFDFDFDFEFEFEFEFFFFFFFFFFFFFFFFC5
:10085000FFFF0000FFFF0001FFFC0100FD0AFBF9A4
:1008600003F50705F7E00E53461EECCCBBB0AFB165
:10087000B3BFCADED9CEE004294962677171767CC4
:100880007666482C12F9DECBBCB2B1B1BBC2C9D579
:10089000DEE5F4F4FBFAFA07FFFF020B1521313B0A
:1008A0003E423F423B38332A29211B171A08FCEAF3
:1008B000D4C5B0A59E9A949AA1A5B0BCC8D1DAE3DC
:1008C000ECF6FCFF0C0F131E1C171421212D323ADD
:1008D0003E42433D3C332E291B16170D080206F7F6
:1008E000F1E8DFD4C9C9C7C4BEC4BEC3C6CED4D91B
:1008F000E5EEF8FD070C141518151619171A19143A
:1009000011160D05FF0C08030F10151B27252A2EA5
:10091000282625211E1C10100E020E010505FCFEC6
:10092000FD00EDF5F0DCD4D6CDCBC4BFC0BFC6C34F
:10093000C2D1D0D6E0E1ECF1FAFC0108110A080EB0
:100940001214151915181E1D1918171923262525F7
:1009500024272530271F1A1B1D160F020406110617
:100960000004FEF1ECEEE8E3E0DCDEE9DEDBD7DDFF
:10097000E6E2DEECEAEBF1F0FFF702000501090B1D
:10098000010CFE0607000100FF03FFFE090A010A31
:100990000E1B1A1D181A2F25221D1A222615211B7F
:1009A0000C141810130F0C06F807F6F6E5E5DAC973
:1009B000D9D1C2C3C6C7D5C2BCC0BEC8DFDADFE763
:1009C000EAF8F0F2FA05000311FE1317101B1A20C3
:1009D0001E2616311E1C292D2B1E382F25282C0DC6
:1009E000311B0F17051708120D0C02FD02F8F1EF6D
:1009F000EAE9EEDAD4DFE5E7D9D5E1EADAD5DAE8F3
:100A0000F5F3EFE30102F9F1FF05F4FEFD02EBFD62
:100A1000FCFEF8ECFF0107050A0B0E1827161B1A3F
:100A200016352523180F281820190D1E1E0C0E1917
:100A30000D08F8F9F3F4F7E7F1E4DAD8DCE1CACC11
:100A4000DDDBD4DADAE0D4E8E2EAE6ECFCE909FD41
:100A5000E7F50FF712FF0E0B0B1D121A0A220D1FDE
:100A6000112010213011102D2204240323080B190A
:100A700005141D100A07FE07FAF8E504F0EEE7E892
:100A8000F9F0ECE7E8F3EFE1FAEFEDF101F0F9F15D
:100A900001FEEE02FBFC03F6EBF6F20DFBF7DEF6D1
:100AA000050108F91307141313180F0D16140E1D62
:100AB0000912160A1D0D04FF121707050C02F20990
:100AC000F8EEECE5E7F0EBE2EDDDE7EBEDF8ECE27C
:100AD000DBF3F5E7ECF4F005FEE5FCFBF70C0A05AB
:100AE00005170CF424051012000B010A18150C252B
:100AF0000A131510050E1013010010FE161803FC42
:100B00000E07FFFDFAF0F500FDE5FD03ECF5FFEE45
:100B1000EAFDF6F3F1F7F7F5EAF0FBFBF40902FA68
:100B2000F5F901F9FDF4F6F80EF301F50D0CFB0CE7
:100B3000F6171B0C1118150D08170A1907020A0ED3
:100B40000D07070C0009FCFE0AE7F8EAF5E1F2EEF2
:100B5000E8F5E8E4ECFBF6EEE7ECFBF9FEF3F4F77E
:100B6000F90DF5F8F70D03FD1213F40717F7FE0B57
:100B700006080B07190BFF02051710011D0C0405D1
:100B80000F0A0310020C0911050600F307FEF6FC1C
:100B9000F203F2EEFCE105F8F3FAE604F6F9FAF9ED
:100BA000FDF609F9FAF3F101FFF201F5F40CF1FC9D
:100BB000FCFC0606F40407FF0B0B0AFFFB112401E3
:100BC000F81407001E04041AFF0B0C050C0207FEA4
:100BD000FCFF01F7EEEEF2F5F2F0F4F5E8F7F2EDD6
:100BE000FFF7EBF5FDF304F8EEF8F30EF405090159
:100BF0000CFCFC0808FA0BFD020908F906051006B2
:100C0000F50D0B0DFB0F070E0202080418FD010580
:100C1000020B0C0BED01FDFA08F40CF8F5F8F0FBF3
:100C200005F9FBEF00FDF7FBEF01FA0BF70100FE02
:100C3000F4F903FBEEF301F6FFF300F201FDFB060E
:100C4000F70506FF07070504050C04040D09050B4D
:100C50000808080708FF010806FE0205FAFBF6FD72
:100C6000FFFAF4FBFEF8F8F9FEF9FDFBFEFFFDFAD2
:100C7000FD00FFFE0000FFFEFF00FE00FF00FF0082
:100C8000FF00000004FFF112FCFA0FF706F003006A
:100C9000FF00FD1000FCEE0DF9FB04030A020FF942
:100CA0002107F612E502FD10FBE1FBEF08EAFAF876
:100CB000F509F701F7F6FD061B06FFF3E906F41048
:100CC000051809080EF705EC0AE7FBF404F5EF0830
:100CD000F70BEE17F70E00090B0410EA0DF90CF6EE
:100CE00004E6EE03F90EEF03FF12FB0B0E0007F113
:100CF00008F9FBFBFEF9EEFDFC04FCFE0B0C040105
:100D000003F8F3FE0207000B0601FDFF0901FFFADD
:100D1000FFFD0BF4FEF6FC020404FD0CFA04E904EA
:100D200008FC07FAFEFFFCF5F6F606FBFB03FF03E3
:100D300009FF0200000CFD04FDFEFA0C00020FFF8B
:100D400006F706FCFFFDF0FFFCFCFEF9F9080401C4
:100D50000802FB00F801050600F501F40008FAFDA1
:100D6000FDF9FF03FB05FC0410F908040107FAF480
:100D7000F9070101FD00010201F7FB07FDFAFDF98A
:100D800004FE0807000B01FBFDF5F705FDFDFCFD6A
:100D900005020AFAFD08F9F8FE03FF050201030245
:100DA0000801FDFEF9FD01FDFF0201FAFC00FB0157
:100DB0000101010202F90106FEFD0702FFF7FA0335
:100DC000FE01FFFFF90109FFFD0306FB04FDFF0320
:100DD000F3FD0205FB02F80301FC02FA08F7010526
:100DE000FBF9FF04FFFD0400FDFFFF04FFFF030408
:100DF0000101F90406FEFCFC0002FEFD03F902FEFF
:100E0000FFFE0200FBFAF903FE05FA0402FE07FFEB
:100E1000FE0100FB02FD03000204FB010203FD03CF
:100E2000FDFE03FCFFFE01FCFAFF04FDFDFEFB01DD
:100E3000FD06FE00020100FE01F705FB0404FE06AC
:100E4000FF00FC0402FFFF01FDFEFFF901FFFA01B4
:100E5000FDFD02FB03FEFD03FFFE01010000000299
:100E6000FE010500FE03FE00FE00FFF900FFFFFB90
:100E700002000200FE01FD00FEFCFF0301FFFDFE7B
:100E8000FFFF01FE010302020000FE03FBFD02FF63
:100E9000FDFD0501FFFF000100FDFE0001FF000256
:100EA000FEFFFE03FDFE01FEFFFF0301FEFEFFFF4E
:100EB000FF00FF000100000403FEFFFE000000FE33
:100EC000FB00000001FDFEFFFEFD00FEFE01FE0036
:100ED0000001FF000102FEFF0000020101FF02FF0E
:100EE00000FF01FE00FFFD01FE00FEFF0000FFFF0E
:100EF0000000FFFF00000000FF0000F912EFF118F2
:100F000011E7EC030C21F7F3EF060012CA17339632
:100F10003A6DCB97E1116A2AE0E6D0051B01C9EED4
:100F20004850DC9CD3FA203EF5EE1FF6CFE625357F
:100F3000E0CAFE033531E2EB13E6C1E9314302FEBC
:100F40000FEEFEDAAE03410FF8112F10D4DAE3EC06
:100F50001909E7363EE7CFE71207E301081834F135
:100F6000C90A0DD3E3113124FA00F7FE01BBCE33D9
:100F700027FC0D1C16F5DAD5EB1020EA034607D541
:100F8000E2F30E00F6030A310EC8EB19EDD7031990
:100F9000301AF1EAF40CEAC00B320206101408EF22
:100FA000D0DC092302E92826E6E6ECF61001F80673
:100FB0002124DFCF0A03E6FF09162C08E4ED02FE28
:100FC000D3E82C15000B03080AE3D3F51817F20633
:100FD00025FDE9F2E90415F6FA182600CFEC08F42D
:100FE000FC0C032120EAE4FE04EDDD0D20060A02DC
:100FF000F910FFD4E80F1803F9120EF2F2EDF11810
:1010000009EE0B1F10E7DDF9FEFD0C010C2600E1D7
:10101000F603F8E9F617130A06F00113E8DC0412E8
:101020000B00FF0D02F5F1E8081DF6FA1610F9E5C0
:10103000EBFC020904FE1A17EBE900FCF4F40314BC
:10104000110AF5F00F01DEF70E0C06FC0107FFF2A6
:10105000EAF71D0BF1080E00F7ECF1010706FB0E95
:101060001EFDE5F7FFF8FBFA06140FFDEEFE0CED92
:10107000ED0A0B0A03F70005FCF0EF0C16FBFE0C63
:1010800000FCF7EBFB0B06FDFF170FEDF2FCF60083
:1010900000FB0D1404F3F507FDEC000B090AFBF24D
:1010A0000206F7F1FE1208FC0602FAFEF1F0090B47
:1010B000FFFC0813FDF0F9F7FC06FB00140BF7F337
:1010C000FE04F7F806060A05F2F809FDF3FA080D22
:1010D000020102FBFFFBECFF0F03FD010B07F7F61C
:1010E000F8F90602F90A11FDF4FA0000FAFF040704
:1010F0000BFBF00403F6F8020B0701FEFDFF00F105
:10110000F30B0B0000030500F8F8F90306F8000FD5
:1011100006F6F9FC0001FDFF040904F3FA06FAF8EB
:10112000FF050906FEFAFD02FAF1010C03000200B8
:1011300003FEF6F8FF08FFF90809FBFAFBFB0302C0
:10114000FE010506FBF60300F9FD01040902FBFBA5
:10115000FFFFFAFB04040001FFFF01FDFBFF020299
:10116000FDFF0200FEFFFE0001FFFF000000FFFF89
:1011700000FFFFDCE6550BE0FC05F4FD08FD04056F
:10118000FA05FD0006F6FBFE060804F5FBFEFE016F
:101190000803FC04F7FF03FDFEFF0400FEFFFF0150
:1011A000FFFC00000200FF00FDFF0101FFFFFDFC4E
:1011B000FF02030300FEFAFBFE020304FE00FD0231
:1011C000FF01FF01FE00FEFFFEFE3CC1BB0C104212
:1011D0002E0FE4D7EE1303EA0B14EEFD17FCECFA26
:1011E000F1FA0AF810110105F5F3010D07F8F5FC05
:1011F000FE00040302FE00FCF7F904060300F803F6
:1012000003FE03FEFD02000200FEFAF8FEFF0003EB
:1012100001FCFBFEFE05050200FEF9F8000705FED5
:10122000F6F6FE06090605FBFAF007D1D54D40FBA0
:10123000CAF510E90C1FF0F9100CFAD1DD0F1D1BD7
:10124000180DF3E4EBF70B101506F7E7F50A08069F
:10125000FEFEFA0904F4F6FF0202030605FDFAF0A9
:10126000FC070C07F8F1F306030C01FEFCFE02017B
:10127000FBFBF9F2FA040D0A0CFC00EE05BFE335A6
:101280001B09230BD608FF10E3DCEF211C0A08EC36
:10129000FF070DF0F4FE0D1010D9CCFB182E18002E
:1012A000E8F112F8F3EF010507100B06F6F4E5FC80
:1012B0001417FDF6F707F4E5FB1E1500EBE805FE35
:1012C000230DE1F40EEFE70F15FD000B0701E4EC31
:1012D00019FBFF040005FA10FFF6F302F904FBE422
:1012E00000140617FFD9EEFA121A0EFA0AF8F5FDE5
:1012F000E4F3111B10F9E9E91119F903FEF3FEF704
:101300000403ECF815150D00F703F1F1EAFD0819D7
:101310002002E7DAEBFE090A110C12FEF6F50302D1
:10132000F3F907F4E91606030E04F8E4F3060909D5
:101330000AF3F00606131208F9F5E5E40110130F9D
:101340000DFDE4D9F50F131510F8F4F1FCF8EFFCDE
:1013500010120E07FFEFE706FD110A01FCF9F5FA7E
:101360000AF4FF0C0D0704E8E50204040E0CFCEC83
:10137000F3071307F4F000FF040F080FFFF3F60163
:10138000FD02FAFAFD02100905EDEDFD0AFAFC0571
:1013900001090D08F3E9EBFF0C090801090CFCFA3F
:1013A000F0F4010A0F03F9F2E8F713090204060149
:1013B000ECEE02110AFEFBFC0B070A05F5FAFB0432
:1013C000FBF7040C070005F7EAEEEFF60712161319
:1013D0000BF7F3F6F7FC01010405FD01F8040BFE21
:1013E000FBFDFAF2F7070A090900FF01FAF4020F00
:1013F0000DFDF5F1F0FF0F0E0D0BF7E6E1FA0F1002
:101400000801FCF70506FBFBF7F4FD030C161607B5
:10141000FBEEEFFAFC050809FDFEFBF6F5FA0609FE
:101420000A0400FAF6FB0303FFF7F1F80710140CA7
:10143000FEF1ECF800030C0400FFF8FD0706FA05C6
:101440000700FAF8FB000803F8F2F2F4F800090EBE
:10145000141507F8F6F3FB0701000603FFF9F9FB83
:1014600005080405FCF1EEFB060B0CFCF3FF050080
:101470000102FC02070602FDFBFCF8FC040704FB6A
:10148000FDFD010601FE00FBFD00FE03FCFC030266
:10149000070602FBFFFDF4EEEEFB0C111109F4F15F
:1014A000FB0407080701F7FE0202040100FDF8F63D
:1014B000FAFC050D08FFFDF6FB02FDFFFF01070624
:1014C000FDFBFD0203020301FDF8FAFFFFFBFB0237
:1014D000090D08FEF7F5F6F9F9FE080F0F07FEF7FC
:1014E000F6FD00FFFE010301FEFCFEFE020300FD0F
:1014F000FC020503FEFAFD0202010202FFFDFBFAF7
:10150000FE00FFFAFB02060705FFF9F8FD010203E2
:10151000020100000000FFFDFE0000010000FFFED0
:10152000FDFEFF01000000FFFFFF00FFFFFF0000C6
:1015300000FFFFFFFFFFFF0000000006F818D218B1
:101540004EBF88B70E507F73532905DFC0A8999608
:101550009AADBED800100D121F354759636B6A66ED
:101560005A4A351E08EEDED3C4B3A59B9796999FC1
:10157000A8B4C1D3DDF50C0E101B30485D6C757737
:10158000736B5D4C38240CF8EDDCC8B6AAA29F9FA3
:10159000A2A8B1BCCCD7E5010B0A0F20364C5D6880
:1015A0006D6B65594B38250FF9EDDECBB9ABA39FB9
:1015B0009EA1A6AFB9C7D7E1FA0C0D101B30465952
:1015C000666E6E6A6052412E1A02F3E6D4C0B1A76D
:1015D000A1A0A1A6ADB7C2D2DCEF070C0C14263B2C
:1015E000505F686C6962564633210AF7EBDAC7B67A
:1015F000AAA3A1A2A6ABB5C0CFDBE8010D0C101EBB
:10160000334859646A6964594B392712FDF0E2CFB7
:10161000BCAFA7A3A2A5AAB3BDCAD8E2F80A0C0E14
:10162000192D4153606768645A4D3D2A1701F2E64F
:10163000D5C2B3AAA5A4A7ACB3BDC9D8E2F4090E1C
:101640000E1525394B596265625B4F412F1D08F518
:10165000EADBC9B8ADA7A5A6ABB1BBC5D4DFED0425
:101660000D0D111F3144545E63625D5345352310E7
:10167000FBEEE2D1C0B2AAA7A7AAB0B8C2CFDCE8FD
:10168000FD0B0C0F192A3D4D5960615D55493928F4
:101690001602F2E7D8C7B8AEA9A8AAAFB6C0CBD990
:1016A000E3F6080B0C14243647555D5F5D574C3E3E
:1016B0002D1C09F6EADECEBEB2ABA9AAAEB5BEC8F5
:1016C000D6E0F0030A0B101E2F414F595D5D574EB7
:1016D00041322110FEEFE4D6C5B7AEAAA9ACB2BA2A
:1016E000C4D0DCE9FC07090E192A3C4B565D5E5B51
:1016F000534739281704F3E7DBCBBCB1ABA9ABB038
:10170000B7C0CCD8E3F603070A1423354551595C1A
:101710005A544A3D2D1C0BF9EBE1D3C3B6AFABAC29
:10172000B0B6BFC9D5E0F00005080F1C2C3B464EF3
:1017300051514C44382B1D0EFFF2E9DFD3C8C1BE16
:10174000BEC0C5CCD4DDE5F0FC020509111C273074
:10175000373A3A38322B22180D03F9F2ECE4DCD692
:10176000D3D2D4D7DBE0E6ECF3FB00020409101778
:101770001D21242423201C16100A04FEF9F5F1ED86
:10178000E9E7E6E7E8EBEEF1F4F8FCFF0001030619
:10179000090C0E0F0F0F0D0C0907040200FEFCFBD5
:1017A000FAFAF9F9FAFAFBFCFDFEFEFFFF000080F1
:1017B000C0408080C0408080C0408080C040800C9D
:1017C0000D080B110E13000102040305060707069E
:1017D000020503040F1012010000020000030004C0
:1017E000000500000000240027002A00000000007F
:1017F000250028002B0000000000230026002900FF
:1018000004040404040404040202020202020303A6
:1018100003030303010204081020408001020408AE
:10182000102001020408102000000007000201003F
:10183000000304060000000000000000E015A730CF
:101840008731D138D91511241FBECFEFD8E0DEBFC4
:10185000CDBF11E0A0E0B1E0EEE0F9E702C00590F5
:101860000D92A634B107D9F717E0A6E4B1E001C0A4
:101870001D92A031B107E1F718E1C4E4D8E104C03A
:101880002297FE010E943F3CCC33D107C9F70E944A
:1018900028390C947A3C0C940000A0E0B0E0E3E519
:1018A000FCE00C944B3CEC01A880B980CA80DB8042
:1018B000A114B104C104D10441F484E2A82E89ED3D
:1018C000B82E8BE5C82E87E0D82EC601B5012DE1D4
:1018D00033EF41E050E00E94223C27EA31E440E04F
:1018E00050E00E94AE3B7B018C01C601B5012DE1A9
:1018F00033EF41E050E00E94223CCA01B9012CEED6
:1019000034EF4FEF5FEF0E94AE3B6E0D7F1D801FE7
:10191000911F97FF04C061507040804090486883D9
:1019200079838A839B839B01AC015F77B901CA01EC
:10193000CDB7DEB7EAE00C94673C0E944D0C0895E9
:1019400080E091E00E944D0C089560930001709337
:1019500001018093020190930301089560E070E01B
:1019600020C0F901E05FFE4F8081480F511D2F5FBD
:101970003F4F26173707ACF3FB01E353FD4FCA0176
:1019800023E0959587952A95E1F78083FB01ED5239
:10199000FD4F4770507040836F5F7F4F6630710519
:1019A00029F040E050E020E030E0E3CF08958F924E
:1019B0009F92AF92BF92CF92DF92EF92FF920F93DE
:1019C0001F93CF93DF9370E0FB01E05FFE4F9081A8
:1019D000892E9924C0E0D0E050E020E030E0B3ED63
:1019E000AB2EB2E0BB2EA60EB71EADECCA2EA2E007
:1019F000DA2EC60ED71E90E0BC01660F771F680F67
:101A0000791F660F771F66527D4F41E0E42EF12C5F
:101A1000012D112D40C0F5014081C901840F911D98
:101A20008031910524F04051420F52E007C00897E1
:101A300024F04850420F51E001C0420FF60180816E
:101A4000FB01E50FF11DE80FF11D808190E002C060
:101A5000959587954A95E2F780FF0DC0D801C7019B
:101A6000022E04C0880F991FAA1FBB1F0A94D2F729
:101A7000C82BD92B0EC0D801C701022E04C0880F75
:101A8000991FAA1FBB1F0A94D2F780959095C8236F
:101A9000D9232F5F3F4F281539050CF4BCCFCE0159
:101AA000DF91CF911F910F91FF90EF90DF90CF903A
:101AB000BF90AF909F908F9008956F927F928F927A
:101AC0009F92AF92BF92CF92DF92EF92FF920F93CD
:101AD0001F93CF93DF933A0170E0FB01E05FFE4F6D
:101AE0009081892E992430E040E050E0F3EDAF2E54
:101AF000F2E0BF2EA60EB71E90E0EDECCE2EE2E097
:101B0000DE2EC60ED71EEC01CC0FDD1FC80FD91F6D
:101B1000CC0FDD1F11E0E12EF12C012D112D4CC059
:101B2000F5012081CA01820F911D8031910524F0B9
:101B30002051240F32E007C0089724F02850240FCA
:101B400031E001C0240FC301042E02C09595879592
:101B50000A94E2F7632F70E080FF16C0F6018081DF
:101B6000FB01E80FF11DEC0FFD1FE652FD4FD80100
:101B7000C70104C0880F991FAA1FBB1F2A95D2F75F
:101B80002081282B208316C0F6018081FB01E80FFD
:101B9000F11DEC0FFD1FE652FD4FD801C70104C037
:101BA000880F991FAA1FBB1F2A95D2F78095208105
:101BB000822380834F5F5F4F481559050CF4B0CFE7
:101BC000DF91CF911F910F91FF90EF90DF90CF9019
:101BD000BF90AF909F908F907F906F900895DF920D
:101BE000EF92FF920F931F9396E0699FB00111242B
:101BF0009B0103E0359527950A95E1F7D22E667093
:101C000070E020E030E090E0AC01440F551F480F39
:101C1000591FB3E0440F551FBA95E1F7A1E0EA2E32
:101C2000F12C012D112DFA01ED0DF11DE250FD4FAA
:101C3000808190E0062E02C0959587950A94E2F780
:101C400080FF0CC0D801C701022E04C0880F991F65
:101C5000AA1FBB1F0A94D2F7782B0CC0D801C7016A
:101C6000022E04C0880F991FAA1FBB1F0A94D2F727
:101C7000809578236F5F683011F4D39460E02F5F14
:101C80003F4F2630310579F6872F1F910F91FF9036
:101C9000EF90DF900895DF92EF92FF920F931F93E2
:101CA000CF93DF9396E0699FB00111249B0153E02D
:101CB000359527955A95E1F7D22E362F367060E08C
:101CC00070E0C42FD0E090E0AC01440F551F480FE6
:101CD000591F93E0440F551F9A95E1F781E0E82ED4
:101CE000F12C012D112DCE01062E02C09595879560
:101CF0000A94E2F7ED2DF0E080FF12C0E40FF51F2B
:101D0000E250FD4FD801C701032E04C0880F991F70
:101D1000AA1FBB1F0A94D2F72081282B208312C050
:101D2000E40FF51FE250FD4FD801C701032E04C098
:101D3000880F991FAA1FBB1F0A94D2F78095208194
:101D4000822380833F5F383011F4D39430E06F5F9B
:101D50007F4F6630710539F6DF91CF911F910F915A
:101D6000FF90EF90DF9008950F931F93CF93DF9331
:101D70008091BF038F5F8093BF038150833010F049
:101D80001092BF038091BF038823B1F5C5EDD1E068
:101D900060E070E003E210E08881882339F1FB0104
:101DA000E954FC4F8081882309F1609FF001619F15
:101DB000F00D709FF00D1124E154FE4F2285338504
:101DC0004485558586819781A085B185820F931FB3
:101DD000A41FB51F82839383A483B58382819381DB
:101DE000A481B58182879387A487B5876F5F7F4F72
:101DF000A3966530710581F6DF91CF911F910F9108
:101E0000089508950895BF92CF92DF92EF92FF92C6
:101E10000F931F93CF93DF93B82E10E000E0C0E044
:101E2000D0E081E0C82ED12CE12CF12C3BC01F5F0B
:101E3000173010F00F5F10E0E02FF0E0E352FC4F9E
:101E4000828190E0012E02C0959587950A94E2F771
:101E500080FF0DC0D701C601022E04C0880F991F54
:101E6000AA1FBB1F0A94D2F7482B592B0EC0D701CB
:101E7000C601022E04C0880F991FAA1FBB1F0A9417
:101E8000D2F780959095482359232F5F3F4F26170F
:101E900037076CF28B2D6C2F0E945D0D2196C6309A
:101EA000D10559F0FE01E05FFE4F8081682F70E0A0
:101EB00040E050E020E030E0EACFDF91CF911F9189
:101EC0000F91FF90EF90DF90CF90BF9008950F9308
:101ED0001F93CF93DF93C82FD0E0CE018370907013
:101EE000892B09F05DC00FB7F89460916E02709174
:101EF0006F0288E06030780708F48EC010E020E0C0
:101F000080E090E004C0660F771F881F991F2A9514
:101F1000D2F722E330E040E050E00E94AE3B3EE0EA
:101F200096958795779567953A95D1F720E130E0BA
:101F3000211B310904C0660F771F881F991F2A953E
:101F4000D2F760937C0270937D0280937E0290931F
:101F50007F020FBF2FB7F89480918502909186027F
:101F6000A0918702B09188028093700290937102D1
:101F7000A0937202B09373022FBF80917002909170
:101F80007102A0917202B0917302809378029093D3
:101F90007902A0937A02B0937B0281E0809384025D
:101FA000CF70D070CD2B09F03DC00FB7F894609181
:101FB0006E0270916F0288E06030780780F110E067
:101FC00020E080E090E004C0660F771F881F991F13
:101FD0002A95D2F724E630E040E050E00E94AE3B84
:101FE0002EE096958795779567952A95D1F720E10C
:101FF00030E0211B310904C0660F771F881F991F2D
:102000002A95D2F760937C0270937D0280937E02C2
:1020100090937F020FBF06C018E028E071CF18E050
:1020200028E0CFCFDF91CF911F910F910895EF92CC
:10203000FF920F931F93F82EE62E042F122F0E946B
:10204000EF0D282F112371F081E090E0A0E0B0E0C7
:1020500004C0880F991FAA1FBB1F0A95D2F7422FF1
:10206000482B0EC081E090E0A0E0B0E004C0880FF3
:10207000991FAA1FBB1F0A95D2F7482F40954223EC
:102080008F2D6E2D0E944B0E1F910F91FF90EF90A0
:102090000895FF920F931F93F82E00E00CC08F2D30
:1020A000602F412F20E00E9417101F5F1630B9F7F4
:1020B0000F5F003211F010E0F2CF1F910F91FF90EF
:1020C00008950F931F93CF93DF938C01EB016D3F26
:1020D000710554F46A3F710564F4663F710549F077
:1020E000683F7105A9F405C0CB018E5F904002974F
:1020F00078F40B581F4FD801ED91FC910557104013
:10210000A081B1812D913C91CF016C2FF9010995EE
:10211000C63FD10511F4F80116A2DF91CF911F91AE
:102120000F91089586E491E068EF70E00E946110DD
:1021300008958F929F92AF92BF92CF92DF92FF92BB
:102140000F931F93CF93DF93EC014B015A01F22EB3
:1021500081E0F82671F0CB58DF4FE881F981C5574F
:10216000D040A081B1812D913C91CF0160EFF90168
:10217000099500E010E045E7C42ED12CCC0EDD1E01
:1021800012C0F601A081B181ED91FC9111979501EA
:10219000200F311F0190F081E02DCD01D9016C910C
:1021A00009950F5F1F4F0815190558F3FF2071F0AF
:1021B000CB58DF4FE881F981C557D040A081B1816C
:1021C0002D913C91CF0167EFF90109951EA2DF9196
:1021D000CF911F910F91FF90DF90CF90BF90AF9064
:1021E0009F908F9008950F931F93CF93DF93EC01EF
:1021F0008C010B581F4FD801ED91FC91A081B1814A
:1022000014962D913C911597CF01F9010995892BD1
:1022100009F4CAC1D801ED91FC91A081B181169653
:102220002D913C911797CF01F9010995482F2DA5C4
:102230003EA52115310509F0FBC088A72DA127FF78
:10224000B9C1243F09F4B6C1253F09F4B3C1293F00
:1022500009F4B0C12D3F09F4ADC1822F90E0203FB9
:1022600028F4807F90708038910591F08039910535
:1022700079F0803B910561F0803A910549F0803D0D
:10228000910531F0803E910519F0803C910541F4B3
:1022900047FD06C028A749A781E090E09EA78DA72B
:1022A00028A527FF0FC0243F69F0253F59F0293F9B
:1022B00049F02D3F39F0822F90E0203F28F4807FB5
:1022C000907002C080E090E0813F910509F46CC0FD
:1022D000823F91054CF5803B910509F468C0813B34
:1022E00091056CF48039910509F461C0803A91053B
:1022F00009F45DC08038910509F0E5C058C0803D03
:10230000910509F451C0813D91052CF4803C910563
:1023100009F0D9C049C0803E910509F448C0803F0A
:10232000910509F0D0C048C0883F9105D1F0893FA0
:1023300091055CF4833F9105B9F1833F9105BCF1B0
:10234000863F910509F0BFC00CC08A3F91050CF48F
:10235000BAC08D3F91052CF08E5F9040029708F037
:10236000B2C027FF0FC0243F69F0253F59F0293F35
:1023700049F02D3F39F0822F90E0203F28F4807FF4
:10238000907002C080E090E099AB88AB1FA61AAABB
:102390001BAACC58DF4F81E08883C457D0401EA6CB
:1023A0001DA61CA61BA601C182E090E002C083E02E
:1023B00090E09CA78BA707C080E490E09CA78BA728
:1023C0001DA280EF8CAB2DA53EA58BA59CA50197EA
:1023D0002817390708F4E4C088A587FF12C0843F96
:1023E00081F0853F71F0893F61F08D3F51F0282FDA
:1023F00030E0803F20F4C901807F907004C0C901A3
:1024000002C080E090E099AB88AB88A58F708F5FA9
:102410008FA789A58AAB8BA59CA5039719F48AA5DC
:102420008BAB01C01BAA1EA61DA61CA61BA612C014
:1024300087FF34C08D3F38F48A3F38F4873F79F006
:10244000883F61F502C08E3F48F148AB19AA1AAA2D
:102450001BAA1FA6CC58DF4F81E08883A6C08CA999
:10246000803F89F5FE01E20FF31F44AB2F5F3F4F22
:102470003EA72DA780EF90E099AB88AB2AAB8EA545
:102480008BAB1FA6CC58DF4F81E08883C457D04068
:102490001EA61DA61CA61BA61DA287C088A5FE0100
:1024A000E20FF31F803F11F444AB01C040A72DA5FC
:1024B0003EA58BA59CA501972817390708F470C085
:1024C00088A5803F31F41EA61DA61CA61BA61DA232
:1024D0006BC087FF12C0843F81F0853F71F0893F58
:1024E00061F08D3F51F0282F30E0803F20F4C9018A
:1024F000807F907004C0C90102C080E090E099AB79
:1025000088AB8038910599F08039910581F0803B46
:10251000910569F0803A910551F0803D910539F0BF
:10252000803E910521F0803C910509F046C088A5C8
:102530008F708F5F8FA789A58AAB8BA59CA503970A
:1025400019F48AA58BAB01C01BAA1EA61DA61CA64A
:102550001BA6CC58DF4F81E08883C457D04088A9A0
:1025600099A9803B9105B1F0813B910554F48039E4
:10257000910581F0803A910569F08038910569F400
:1025800009C0803D910531F0803E910519F0803CF5
:10259000910519F488A58DA301C01DA281E005C095
:1025A0002F5F3F4F3EA72DA780E0DF91CF911F9176
:1025B0000F91089580E090E059CE1FA6BCCFFC019A
:1025C00080A991A9813F910509F4BCC0823F910582
:1025D0004CF5803B910509F464C0813B91056CF496
:1025E0008039910509F446C0803A910509F477C015
:1025F0008038910509F0D6C03AC0803D910509F4B4
:102600007AC0813D91052CF4803C910509F0CAC047
:1026100075C0803E910509F447C0803F910509F0DF
:10262000C1C077C08A3F910561F18B3F91058CF461
:10263000833F910509F4A0C0833F91050CF485C048
:10264000863F910509F4A1C0883F910509F0AAC011
:1026500014C08C3F9105E9F08C3F9105B4F08E3F9A
:102660009105D9F08F3F910509F09CC095C020815C
:10267000318137C02281338134C0008CF18DE02D4F
:1026800087C0028CF38DE02D83C0048CF58DE02D86
:102690007FC0068CF78DE02D7BC000A0F1A1E02D5E
:1026A00077C0268137811DC02485358521153105E8
:1026B00009F478C063A970E06F7770707695762F13
:1026C00066277795679582A990E08F779070682B41
:1026D000792B6050704287A5F901099508952481EE
:1026E00035812115310509F45DC087A562A943A98B
:1026F000F901099508952285338502C02085318529
:102700002115310509F44EC087A562A9F901099583
:102710000895468557854115510509F443C093A98D
:1027200080E022A9622F70E09F012C5C3F4F682B54
:10273000792B6134710510F060E470E0C901FA0191
:10274000099508952089318919C042895389411515
:10275000510541F183A990E08F7790709695982F5D
:1027600088279795879522A930E02F773070822BA4
:10277000932BFA010995089524893589211531058E
:1027800089F082A9F901099508950688F789E02D55
:10279000309741F00995089502A0F3A1E02D3097FC
:1027A00009F009950895DF92EF92FF920F931F931E
:1027B000CF93DF93EC017B01142FD22E0150003117
:1027C00018F46038710514F41EA243C0613E71050F
:1027D000B4F5602F6F706E298EA1861771F06EA30D
:1027E000CB58DF4FE881F981C557D040A081B18136
:1027F0002D913C91CF01F9010995CB58DF4FE8812C
:10280000F981A081B1811F772D913C91CF01612F7A
:10281000F901099580ECE816F104D9F080EDE8168D
:10282000F104B9F0E881F981A081B1818FE7D82264
:102830002D913C91CF016D2DF90109950AC0663F9C
:1028400071053CF06F3F710509F01CF4CE010E9448
:102850006110DF91CF911F910F91FF90EF90DF906A
:102860000895EF92FF920F931F93CF93DF93EC01A4
:102870008CA180FFF1C0382F369509F4EDC068A90E
:1028800079A9CB01805890408136910508F50FA5B4
:102890008FA1081719F020E0882309F421E0832F85
:1028A00090E08230910539F08330910541F0019735
:1028B00009F0D2C007C0222309F4CEC003C02223EE
:1028C00009F0CAC0CE014AA92BA90E94D313C4C0E3
:1028D000663F710549F1673F7105ACF4613F7105D1
:1028E00009F490C0623F71052CF4603F710509F056
:1028F000B3C01EC0623F710509F447C0633F710554
:1029000009F0AAC028C06D3F710544F46A3F710503
:102910005CF4683F710509F09FC006C0CB018E5F73
:102920009040029708F098C0CE010E94611094C0B8
:102930009BA980E02AA9622F70E0682B792B613473
:10294000710510F060E470E0CE01E496AE0121E084
:102950000E94991081C00AA935E7E32EF12CEC0EF4
:10296000FD1EF701A081B181ED91FC9111970190BD
:10297000F081E02DCD0163EF0995F701A081B181D0
:10298000ED91FC91119710E035C00BA910E0169560
:10299000102F0027179507958AA990E0082B192B6F
:1029A00095E7E92EF12CEC0EFD1EF701A081B18117
:1029B000ED91FC9111970190F081E02DCD0162EF36
:1029C0000995F701A081B181ED91FC911197B801B2
:1029D0006F7770700190F081E02DCD010995F701BE
:1029E000A081B181ED91FC911197000F012F001F83
:1029F000110B11950F7710700190F081E02DCD0132
:102A0000602F28C08AA990E08770907014E0880F2A
:102A1000991F1A95E1F71BA91F70182BB5E7EB2E2C
:102A2000F12CEC0EFD1EF701A081B181ED91FC911E
:102A300011970190F081E02DCD0161EF0995F7012B
:102A4000A081B181ED91FC9111970190F081E02D71
:102A5000CD01612F09951EA2DF91CF911F910F919A
:102A6000FF90EF9008950F931F93CF93DF93EC01A6
:102A7000062F613128F50E94F310882309F188A9F7
:102A800099A98039910539F48BA9882321F480E82C
:102A900090E099AB88AB88A999A9009759F0805824
:102AA00090408136910598F49FA18FA5891779F000
:102AB000992369F010E0CE01602F0E94311401C00B
:102AC00010E0812FDF91CF911F910F910895CE01DA
:102AD0000E94DF1211E0EFCFFC0167A10E943315C5
:102AE0000895019709F064C06F5F7F4F09F060C0DF
:102AF0008EEE96E09093BC018093BB01109247014B
:102B000010924601109249011092480110924B0117
:102B100010924A0110924D0110924C0110924F01F7
:102B200010924E01109251011092500110925301D7
:102B300010925201109255011092540110925701B7
:102B400010925601109259011092580110925B0197
:102B500010925A0110925D0110925C0110925F0177
:102B600010925E0110926101109260011092630157
:102B70001092620110926501109264011092670137
:102B8000109266011092690110926801E3EDF1E084
:102B90001082B39682E0E53AF807D1F781E992E036
:102BA0006DE370E00E94302A8FEA92E00E94572C79
:102BB000089580E090E06FEF7FEF0E947115089517
:102BC00081E090E06FEF7FEF0E94711508951F93F1
:102BD000182F8091A703882339F0812F90E083700C
:102BE0009070892B19F50AC08091B503212F30E030
:102BF000882371F023703070232B21F48FEA92E048
:102C000061E00FC060918E036E5F8FEA92E015C0A5
:102C100023703070232B51F460918E036E5F8FEA26
:102C200092E00E94A52C112329F009C08FEA92E0BE
:102C300060E003C08FEA92E067E00E94A52C1F913C
:102C400008950F931F93CF93DF93C0E0D0E0082F38
:102C500010E080919303882389F0C330D105F4F00C
:102C6000CE018350682FA8010C2E02C055954795C0
:102C70000A94E2F741708FEA92E00EC0C330D105AA
:102C80006CF4A8010C2E02C0559547950A94E2F702
:102C900041708FEA92E06C2F0E94EE2C2196C63094
:102CA000D105B9F6DF91CF911F910F910895FF9251
:102CB0000F931F9386E491E00E946C158091BF03EF
:102CC0008F5F8093BF03813428F01092BF0380E0B0
:102CD0000E94670F8FEA92E063E00E94182D88231C
:102CE00039F48FEA92E065E00E94182D8823B1F054
:102CF00080918E03282F30E0223031051CF020E037
:102D000030E002C02F5F3F4F20938E0386E491E0B6
:102D100060EB70E04DE001E00E94D3138FEA92E097
:102D200064E00E94182D882339F48FEA92E066E06F
:102D30000E94182D8823B1F080918E03282F30E057
:102D40002115310519F422E030E002C02150304055
:102D500020938E0386E491E060EB70E04DE001E0AB
:102D60000E94D31360918E036F5F8FEA92E00E94FE
:102D7000A52C10E0FF24F3948FEA92E0612F0E94CB
:102D8000182D882339F08FEA92E0612F0E942C2DB4
:102D9000F092EB038FEA92E0612F0E945A2D482FA8
:102DA0008FEA92E0612F0E94EE2C8FEA92E0612F71
:102DB0000E94712C8823C9F08FEA92E0612F0E9453
:102DC000912C412F465F9C0153E0359527955A95EC
:102DD000E1F786E491E060EB70E001E00E94D3133C
:102DE0008FEA92E067E00E94A52C1F5F133021F666
:102DF0008091EB03882379F08FEA92E00E94642DA2
:102E0000282F86E491E060EB70E04EE001E00E9444
:102E1000D3131092EB031F910F91FF900895882315
:102E200009F445C0282F209523708695869581301A
:102E300051F0813028F08230E9F08330C1F51FC0B5
:102E400060FD07C013C0862F90E083709070892BBF
:102E500069F0622F70E080E090E00E946F3A6115A7
:102E600071058105910511F491E001C090E0109287
:102E7000B6031EC0862F90E08770907004C0862F26
:102E800090E08F709070892B69F0622F70E080E085
:102E900090E00E946F3A611571058105910511F46A
:102EA00091E001C090E081E08093B60301C090E022
:102EB000892F089581E992E00E94292B81E0809377
:102EC000A60308953F924F925F926F927F928F92E6
:102ED0009F92AF92BF92CF92DF92EF92FF920F93A9
:102EE0001F93CF93DF930E947231AB01BC0181E944
:102EF00092E00E94C62A8FEF80939903B1EDCB2E0A
:102F0000B1E0DB2E662477244301AA24BB24A3E28C
:102F10004A2E512CD60114968C911497882309F4CB
:102F2000B3C0F501EC56FC4F308012968C9112978D
:102F30001996ED90FD900D911C911C97882381F5B9
:102F4000A49CE001A59CD00DB49CD00D1124C154CB
:102F5000DE4F8A819B81AC81BD818E159F05A007C4
:102F6000B107D0F48A819B81AC81BD819D0144274A
:102F70005527D601ED91FC91E20FF31FE4912A81D0
:102F80003B814C815D818E859F85A889B989820F9F
:102F9000931FA41FB51F54C0E6011C82E0E054C07B
:102FA000A49CF001A59CF00DB49CF00D1124E154FB
:102FB000FE4F82819381A481B581E816F9060A0744
:102FC0001B07A8F482819381A481B581E6012D813C
:102FD0003E814F815885820F931FA41FB51F8E1904
:102FE0009F09A00BB10B82839383A483B583A49C18
:102FF000B001A59C700DB49C700D112461547E4FDE
:10300000FB0182819381A481B581CD01AA27BB27D1
:10301000E601E881F981E80FF91FE491DB011296DE
:103020002D913D914D915C9115971E968D919D919D
:103030000D90BC91A02D820F931FA41FB51FEB0113
:103040008A839B83AC83BD832E2F332727FD309546
:10305000F501E656FC4F808190E028273927832D23
:1030600090E0FC012E9FC0012F9F900D3E9F900D80
:103070001124892F990F990BAA2797FDA095BA2F94
:10308000680E791E8A1E9B1E0894A11CB11C43E287
:1030900050E0C40ED51E56E0A516B10409F03ACF93
:1030A000A401930164E0220F331F441F551F6A954A
:1030B000D1F7C901DF91CF911F910F91FF90EF9050
:1030C000DF90CF90BF90AF909F908F907F906F9048
:1030D0005F904F903F9008950F931F93CF93DF938E
:1030E000082F8A3010F460E013C08FEA92E060E0AD
:1030F00041E00E94EE2C8FEA92E061E041E00E9404
:10310000EE2C8FEA92E062E041E00E94EE2C61E05A
:10311000015087EF9FEF689F102D1124100FC0E022
:10312000D0E08FEA92E0612F40E00E94EE2C8FEA1F
:1031300092E00E94822F66E970E080E090E00E94B9
:1031400095358FEA92E0612F41E00E94EE2C8FEAE4
:1031500092E00E94822F66E970E080E090E00E9499
:1031600095352196C330D105E1F6DF91CF911F91BE
:103170000F9108950F931F93182F8091BB01909189
:10318000BC0142E15AE760E070E00E949D37109276
:103190006D0110926C0110926B01109274011092EB
:1031A000730110927201109271011092BA01109283
:1031B00077011092760110927501109278011092A9
:1031C000790103E000936A011093BE01812F0E94F0
:1031D0006C188EEB91E2909349018093480181E055
:1031E0009FE0909347018093460188E694E2909394
:1031F0004D0180934C0182E09FE090934F018093BA
:103200004E0183ED99E190935501809354018AE535
:1032100097E190935F0180935E018BEC99E190932D
:1032200061018093600186EC99E190936301809342
:1032300062018FEB99E190936501809364010093A3
:103240006A011F910F9108950F931F930FEA12E0E7
:10325000C80160E041E00E94EE2CC8010E94822F6C
:1032600066E970E080E090E00E949535C80162E078
:1032700041E00E94EE2CC8010E94822F66E970E0B6
:1032800080E090E00E949535C80161E041E00E9435
:10329000EE2CC8010E94822F66E970E080E090E089
:1032A0000E949535C80163E00E94A52CC8010E94C8
:1032B000822F66E970E080E090E00E949535C801B9
:1032C00067E00E94A52CC8010E94822F66E970E089
:1032D00080E090E00E949535C80160E00E94A52C36
:1032E000C80160E040E00E94EE2CC80161E040E0CF
:1032F0000E94EE2CC80162E040E00E94EE2CC80162
:103300000E94822F1F910F9108950F931F93082FF2
:1033100010E08FEA92E0612F0E94A52C68EC70E02B
:1033200080E090E00E9495358FEA92E00E94822F23
:103330001F5F183071F768EC70E080E090E00E9449
:1033400095358FEA92E060E00E94A52C8FEA92E02A
:1033500060E0402F0E94EE2C8FEA92E061E0402F67
:103360000E94EE2C8FEA92E062E0402F0E94EE2C49
:103370008FEA92E00E94822F1F910F910895109280
:10338000A70381E992E00E941D2C089581E992E053
:103390000E94232C089581E992E00E94132C81E081
:1033A0008093A6030895CF93DF93EC0189818D3735
:1033B000E9F58A81882341F41092BE018A818F5FEA
:1033C0008A8386E491E02EC0813009F58FEA92E08D
:1033D00067E00E94A52C8FEA92E00E94822F21E0F4
:1033E00030E0F901E452FC4FDE01A20FB31F8C91D3
:1033F00080832F5F3F4F2F30310599F780918F03E6
:103400000E94030F8FEA92E00E947B2C0FC08A304B
:1034100069F481E08093BD0110926A0186E491E035
:1034200060E170E0AE0120E00E949910DF91CF9141
:103430000895BF92CF92DF92EF92FF920F931F9366
:10344000CF93DF931092B4038091A703882309F4EC
:10345000D8C08FEA92E060E00E94672C882389F14F
:103460008FEA92E060E00E94912C8C010C5E1F4F6D
:1034700015950795159507958FEA92E060E00E94F3
:103480009B2CEC016496D595C795D595C79581E998
:1034900092E00E94552B0C171D073CF008171907E6
:1034A00004F18C179D07ECF006C080179107CCF053
:1034B000C817D907B4F08FEA92E060E00E94802C30
:1034C00010C08FEA92E060E00E94912CBC016C5E1B
:1034D0007F4F759567957595679581E992E00E9494
:1034E000402B8FEA92E061E00E94672C8823A1F1D3
:1034F0008FEA92E061E00E94912C8C010F5F1F4FD8
:1035000095E0159507959A95E1F78FEA92E061E0CD
:103510000E949B2CEC01219685E0D595C7958A9554
:10352000E1F781E992E00E94392C90E00C171D0729
:103530003CF0081719070CF18C179D07F4F006C032
:1035400080179107D4F0C817D907BCF08FEA92E032
:1035500061E00E94802C11C08FEA92E061E00E943D
:10356000912CBC016F5F7F4FB5E075956795BA955B
:10357000E1F781E992E00E94362C8FEA92E062E066
:103580000E94672C882371F18FEA92E062E00E942A
:10359000912C8C0115950795159507958FEA92E06A
:1035A00062E00E949B2CEC01D595C795D595C795F7
:1035B00081E992E00E94BF2A90E00C171D074CF0B1
:1035C000081719070CF48BC18C179D070CF487C1E1
:1035D000CAC0801791070CF482C1C817D9070CF430
:1035E0007EC1C1C08FEA92E062E00E94912CBC01D2
:1035F000759567957595679581E992E00E94BC2A5B
:103600006EC18091B503882309F462C181E992E01B
:103610000E94202C882309F45BC180918E038823AB
:1036200009F050C08FEA92E060E00E94672C882386
:1036300069F08FEA92E060E00E94712C882379F0B3
:103640008FEA92E060E00E94802C09C08FEA92E04D
:1036500060E00E94912C9093AF038093AE038FEAB9
:1036600092E061E00E94672C882369F08FEA92E083
:1036700061E00E94712C882389F08FEA92E061E07A
:103680000E94802C0BC08FEA92E061E00E94912C96
:1036900095958795959587958093B0038FEA92E0ED
:1036A00062E00E94672C882309F055C08FEA92E0FF
:1036B00062E00E94912C95958795959587958093CA
:1036C000B1030DC1813009F00AC18FEA92E060E0D8
:1036D0000E94672C882369F08FEA92E060E00E94E4
:1036E000712C882391F08FEA92E060E00E94802C98
:1036F0000CC08FEA92E060E00E94912C46E0959524
:1037000087954A95E1F78093B4038FEA92E061E0F0
:103710000E94672C882369F08FEA92E061E00E94A2
:10372000712C882389F08FEA92E061E00E94802C5E
:103730000BC08FEA92E061E00E94912C95958795ED
:10374000959587958093B2038FEA92E062E00E949C
:10375000672C882371F08FEA92E062E00E94712C5E
:10376000882309F4BCC08FEA92E062E00E94802CBA
:10377000B6C08FEA92E062E00E94912C9595879501
:10378000959587958093B303AAC080918E038B9DF6
:10379000C0011124EF2CE80E8FEA92E06F2D0E94F9
:1037A000672C10918F03882309F466C080919003E1
:1037B000811709F087C08FEA92E06F2D0E94912C4B
:1037C000AC01CE2DD0E0FE01E05FFE4F8081282FBE
:1037D00030E08B3050F4C601821B930B8A0102C08B
:1037E000159507958A95E2F708C02A5030408A015E
:1037F00002C0000F111F2A95E2F78FEA92E06F2DA9
:103800000E949B2CAC01C05FDE4F8881282F30E0E6
:103810008B3050F4C601821B930BEA0102C0D59590
:10382000C7958A95E2F708C02A503040EA0102C0E5
:10383000CC0FDD1F2A95E2F780918F036E2D0E9439
:10384000D70C0C171D073CF008171907DCF18C1773
:103850009D07C4F106C080179107A4F1C817D907C6
:103860008CF18FEA92E06F2D0E94802C8FEA92E01B
:1038700067E00E94A52C26C08FEA92E06F2D0E947F
:10388000912C9C01EE2DF0E0E05FFE4F8081482FEF
:1038900050E08B3050F4C601841B950BA90102C087
:1038A000559547958A95E2F709C04A505040C9019D
:1038B00002C0880F991F4A95E2F7AC01812F6E2D47
:1038C0000E945D0DF39493E0F91609F05ECF07C0F6
:1038D000FF2403E0B02E1AE0C12ED12C56CFDF9189
:1038E000CF911F910F91FF90EF90DF90CF90BF90FD
:1038F00008952F923F924F925F926F927F928F9294
:103900009F92AF92BF92CF92DF92EF92FF920F936E
:103910001F93DF93CF9300D000D000D0CDB7DEB798
:10392000882E2FEB31E03E832D838AE993E09C8340
:103930008B8350EA452E53E0552EE4E9F3E0FA83F9
:10394000E98347EB242E43E0342E66247724ED816F
:10395000FE818689882309F49FC1882029F0F1E03F
:103960008F1609F099C15FC18091B503882309F4CE
:10397000B2C181E992E00E94202C882309F4ABC1F6
:103980008FEA92E060E00E94672C882309F042C031
:10399000DFB6F894ED81FE816081718180E090E076
:1039A0000E94BD3A7B018C016091AE037091AF0320
:1039B0006F5F7F4F882777FD8095982F0E94BF3AD1
:1039C00020E030E040E85DE30E944B3B9B01AC010E
:1039D000C801B7010E944B3B20E030E040E858E3CB
:1039E0000E944B3B20E030E040E857E40E944B3B14
:1039F0000E94913A23E230E0629EF001639EF00D56
:103A0000729EF00D1124E154FE4F66877787808BFC
:103A1000918BDFBE8FEA92E061E00E94672C8823E1
:103A200059F58091B003282F30E02115310519F4A4
:103A3000F101108203C081E0F101808380E091E018
:103A4000821B930B880F991F880F991FAA2797FD38
:103A5000A095BA2FDC019927882723E230E0629EE7
:103A6000F001639EF00D729EF00D1124E154FE4FA3
:103A700086839783A087B1878FEA92E062E00E94F5
:103A8000672C882309F008C100D000D06091B103F1
:103A900070E080E090E0ED81FE812081318140E0A6
:103AA00050E0EDB7FEB721833283438354839BC03C
:103AB000F201808160E00E94D70C7C019FB6F894EF
:103AC000ED81FE816081718180E090E00E94BD3ACD
:103AD0005B016C010894E11CF11C0027F7FC0095C8
:103AE000102FC801B7010E94BF3A20E030E040E843
:103AF0005DE30E944B3B9B01AC01C601B5010E94F6
:103B00004B3B20E030E040E858E30E944B3B20E094
:103B100030E040E857E40E944B3B0E94913A23E298
:103B200030E0629EF001639EF00D729EF00D112454
:103B3000E154FE4F66877787808B918B9FBE8FEA1B
:103B400092E061E00E94672C882361F5F201808198
:103B500061E00E94D70C9C01009719F4F1011082DA
:103B600003C081E0F101808380E091E0821B930B30
:103B7000880F991F880F991FAA2797FDA095BA2F24
:103B8000DC019927882723E230E0629EF001639EE2
:103B9000F00D729EF00D1124E154FE4F8683978341
:103BA000A087B1878FEA92E062E00E94672C8823A9
:103BB00009F072C0F201808162E00E94D70C00D04F
:103BC00000D0AA2797FDA095BA2FED81FE81208114
:103BD000318140E050E0EDB7FEB72183328343836B
:103BE0005483BC01CD0120E030E040E050E0FFEF25
:103BF000EF2EF12C012D112DE0E1AE2EB12CC12CB8
:103C0000D12C0E94263A80E090E0CB0177276627EE
:103C1000ED81FE81638F748F858F968F0F900F904B
:103C20000F900F9039C08091B503882309F45CC0D0
:103C300081E992E00E94202C882309F455C08FEA84
:103C400092E062E00E94672C882329F48091B303FC
:103C5000E981FA8180838FEA92E061E00E94672C1B
:103C60008823D1F48091B20314C0F201808165E011
:103C70000E94D70CE981FA8180838FEA92E061E0AB
:103C80000E94672C882341F4F201808164E00E9445
:103C9000D70CEB81FC8180830894611C711C2D8101
:103CA0003E812D5D3F4F3E832D838B819C8101960C
:103CB0009C838B830894411C511CE981FA813196C5
:103CC000FA83E9830894211C311CF5E06F16710416
:103CD00009F03DCE11C08FEA92E060E00E94672CAF
:103CE000882309F02CCFE4CE8FEA92E062E00E94B4
:103CF000672C882311F6B9CF26960FB6F894DEBF4D
:103D00000FBECDBFCF91DF911F910F91FF90EF902C
:103D1000DF90CF90BF90AF909F908F907F906F90EB
:103D20005F904F903F902F9008950F931F93CF93E4
:103D3000DF9328E1829F8001112402501D4F90E003
:103D40000196EC01CC0FDD1FC80FD91F63E0CC0F2B
:103D5000DD1F6A95E1F7C250DD4F84E690E00E94D6
:103D60000D31F80181938F01EC17FD07B1F7DF9159
:103D7000CF911F910F9108950F931F93CF93DF93CE
:103D8000082FC4E7D0E010E0FE01859194910E94D5
:103D90000D31AC01802F612F0E945D0D8FEA92E002
:103DA0000E947B2C22961F5F163071F786E090E010
:103DB0000E940D31AC01802F63E00E945D0D82E313
:103DC00090E00E940D31AC0148535F4F802F65E0B9
:103DD0000E945D0DDF91CF911F910F9108955F9229
:103DE0006F927F928F929F92AF92BF92CF92DF920B
:103DF000EF92FF920F931F93CF93DF93682E562E6F
:103E000025E0821711F0482F01C042E0C42FD0E016
:103E1000FE01E056FC4F60821091B40381E992E00C
:103E20000E943F2C682F812F0E940F17882309F4CE
:103E3000E9C08091B603882309F474C086E090E05D
:103E40000E940D31482F50E0440F551FFA01E65DE6
:103E5000FE4F8081918123E230E0C29FF001C39F39
:103E6000F00DD29FF00D1124E154FE4F4C5F5E4FD8
:103E7000DA012D913C91338B228B91838083178AB9
